:100000000AC018951895189518951895189518956B
:100010001895189518958FED8DBFC0ECE0EC4E2E1D
:10002000DD275D2EEEE7F0E0A0E6B0E088278D93B7
:100030003197E9F757D266248FEF81BB8EE187BBFA
:10004000C09AC59AC69AC79AC29AC19AE4E6F0E0E5
:1000500080E490D258E0C895802D86D231965A958A
:10006000D1F704C00C12120C20202020E4E8F0E0AC
:1000700080E580D258E0C895802D76D231965A9589
:10008000D1F704C020201F1F1F1F202011D28CE099
:1000900071D2E8E3F7E004D2E2E0F0E01AD208D24D
:1000A000E8E4F7E0FDD102D2EEE4F7E0F9D1E3E0D5
:1000B000F0E00FD2FDD1EAE0F0E0ABE617D3E4E1E7
:1000C000F0E0ACE613D3EFE0F0E0A7E60FD3EFE00B
:1000D000F0E0A0E10BD3043608F00EC0E9D1EEE564
:1000E000F7E0DED1E3D1E8E3F7E0DAD1C498C398D2
:1000F00085B7806385BF8895C298C0D1BFD180E0A5
:100100008093600080E08093610081E080936900CB
:1001100000916900083010F009F01CC0A1E60C91B4
:1001200042E0EED24C93AAD1009161004091600070
:10013000040FA1E60C93B09B04C081E080936000A3
:1001400003C080E080936000A9E68C918F5F8C9360
:1001500008F4DECFC29A84E690E038D2A4E68C910F
:100160008F5F8C9300916400003408F001C014C0CC
:1001700080E08093640040916B000091610004175F
:1001800010F009F001C0C49A40916C000091610028
:10019000041708F401C0C4988FE711E098D1E0E794
:1001A000F7E07ED1009161000A3008F003C0E4E777
:1001B000F7E076D1A8EAB0E0E1E6F0E037D268D126
:1001C00080E0D2D1E6E7F7E06BD18FE71AE07FD18C
:1001D000EAE7F7E065D1C49904C0E0E8F7E060D150
:1001E00003C0E4E8F7E05CD18091610080936A008D
:1001F00013D1BE98A8E69C9196FF04C0B69B0EC092
:100200009F7B9C93B6990AC089E19F939927DED181
:100210009F91B69903C090649C9301D058CFEFE0B2
:10022000F0E0A7E663D28091670081508093670079
:10023000EFE0F0E0A7E67BE748D2809168008F7797
:100240008093680035D1E8E8F7E02AD12FD1EAE9B8
:10025000F7E026D1BD98A8E69C9195FF04C0B59B18
:100260000EC09F7D9C93B5990AC089E19F93992701
:10027000ADD19F91B59903C090629C934FD0BF9828
:10028000A8E69C9194FF04C0B79B0EC09F7E9C93F0
:10029000B7990AC089E19F93992798D19F91B799FF
:1002A00003C090619C9379D0A8E68C9187FB0EF4F3
:1002B00001C02DC0EAE0F0E0ABE67BE706D2E4E166
:1002C000F0E0ACE67BE701D2EAE0F0E0ABE60ED28C
:1002D000E4E1F0E0ACE60AD240916C0000916B00E2
:1002E000041708F414C0E4D0ECEAF7E0D9D0009188
:1002F0006B0041E0040FACE60C93E4E1F0E0ACE607
:100300007BE7E3D1E2E0F0E0E4D0D2D00895A8E6C4
:100310008C9187FB0EF001C008959CCF80E0809304
:100320006B00C6D0B69906C0809168008068809343
:1003300068000895B59907C084E690E047D1ABE620
:100340008C918F5F8C938FE711E0C1D0EEEBF7E0DB
:10035000A7D000916B000A3008F003C0E4E7F7E093
:100360009FD0A8EAB0E0EBE6F0E060D191D080E069
:10037000FBD0E2ECF7E094D080916B0080936A00B0
:100380004BD000916B00033610F009F001C004C09F
:1003900080E080936B008CD0C5CF80E080936C00B0
:1003A00087D0B69906C08091680080688093680005
:1003B0000895B79907C084E690E008D1ACE68C9127
:1003C0008F5F8C938FE711E082D0E6ECF7E068D086
:1003D00000916C000A3008F003C0E4E7F7E060D059
:1003E000A8EAB0E0ECE6F0E021D152D080E0BCD049
:1003F000E2ECF7E055D080916C0080936A000CD05D
:1004000000916C00033610F009F001C004C080E0D8
:1004100080936C004DD0C5CF84E690E0D7D08FEBB1
:1004200011E055D000916A0042E076D1A6E60C9327
:100430008091660081508093660081E08093670020
:100440004091660000916700041710F009F010C099
:1004500000916600003110F009F001C001C00DC02C
:1004600082E082D0A7E68C918F5F8C9308F4E8CF6E
:1004700082E07AD0EAECF7E013D00895969AEF93F1
:10048000FF93E6E0F0E096D0FF91EF919698089503
:10049000A8EAB0E08D91882311F066D0FBCF0895D3
:1004A000A4D0802D11F060D0FBCF089580EC62C005
:1004B00081E060D014D080E85DC08FE7213039F052
:1004C0008FEB223021F08FE8233009F08FEC810F81
:1004D00051C088EE93E07AD03197D9F7089583E040
:1004E000992774C08AEF90E071D08D9A8C9A8B9A7C
:1004F0008A9A899A889A909885E090E067D0919836
:1005000095989498939A929A919AEF93FF93E0E634
:10051000F0E050D0FF91EF91919855D0919AEF93E0
:10052000FF93E0E6F0E046D0FF91EF9191984BD039
:10053000919AEF93FF93E0E6F0E03CD0FF91EF91CA
:10054000919841D09298919AEF93FF93E0E6F0E072
:1005500031D0FF91EF91919836D088E20BD08EE0A8
:1005600009D086E007D00895909A829505D004D0EE
:100570002AD008959098F9CF859510F4929A01C0E9
:100580009298859510F4939A01C09398859510F4EC
:10059000949A01C09498859510F4959A01C0959805
:1005A000919AEF93FF93E0E6F0E004D0FF91EF9192
:1005B000919808953197F1F70895689462F8089535
:1005C000E89462F8089581E090E000C0EF93FF9313
:1005D000EE27E82BE92B31F0E8EEF3E03197F1F765
:1005E0000197D1F7FF91EF910895C89531960020BA
:1005F0000895000F111F221F331F089500951095B5
:10060000209530950F5F1F4F2F4F3F4F0895019159
:1006100010810EC001911191219130810BC0019187
:10062000108117FF05C03FEF2FEF04C00081112795
:100630002227332737FF03C0E1DF8DE28D93CF936D
:10064000DF93CF92DF92EF92AA24BB24CC24DD2447
:10065000EE2440E2CAE0DD2755E093E38881890F6C
:1006600087FD9F7083FD907F891B89935A95A9F719
:10067000C0DFAA1CBB1CCC1CDD1CEE1C4A9551F72C
:10068000E894EFE0FF2782910ED0EB30E0F71EF008
:1006900068948A2D0CD088278D93EF90DF90CF90AF
:1006A000DF91CF910895982F829501D0892F8F7077
:1006B000805D26F0803309F4089568948D93089541
:1006C000E199FECFEEBB3196089591E001C092E032
:1006D0007B3751F47FB7F894F3DF8D918DBBE29AAD
:1006E000E19A9A95C9F77FBF7727089591E001C0F5
:1006F00092E0E6DFE09A8DB38D939A95D1F7089555
:10070000FF935527F8E0469508F4500F5795479505
:10071000FA95D1F7FF910895FF93881BF9E0001F28
:10072000FA9511F4FF910895881F841B18F4840F23
:100730008894F5CF0894F3CF5757572E4156522E31
:10074000344D472E434F4D0044454D4F0000475315
:100750004D3A3034302038333231373900002120DF
:1007600044454D4F204558504952454420210000F2
:10077000543A00002000432020004F55543A000016
:100780004F4646004F4E200054313D4C4F57202DD0
:100790002054323D4849474800003C54313E202017
:1007A0003C4F4B3E20203C54323E00005432206DE2
:1007B000757374206265203E20543121000054314D
:1007C0003D004320000054323D0020202020000046
:00000001FF
